:03000000020C00EF
:03000300021A03DB
:03000B00021A06D0
:03001300021A09C5
:03001B00021A0CBA
:03002300021A0FAF
:03002B00021A12A4
:03003300021A1599
:03003B00021A188E
:03004300021A1B83
:03004B00021A1E78
:03005300021A216D
:03005B00021A2462
:03006300021A2757
:03006B00021A2A4C
:03007300021A2D41
:03007B00021A3036
:03008300021A332B
:03008B00021A3620
:03009300021A3915
:03009B00021A3C0A
:0300A300021A3FFF
:100C0000787FE4F6D8FD9000007F007E20E4F0A31A
:0A0C1000DFFCDEFA758120020C55AE
:101A3C0006012C034D056E078F09A70B0000000053
:101A4C0000000032006400C8012C015E019001C24C
:101A5C0001FC022E0261029402C702FA032C035FFE
:101A6C00039203C503F8042A045D049004C304F62E
:101A7C000528055B058E05C105F406260659068C5E
:101A8C0006BF06F207240757078A07BD07F008228E
:101A9C000855088808BB08EE09210953098609B9BD
:101AAC0009EC0A1F0A510A840AB70AEA0B1D0B4FEC
:101ABC000B820BB50BE80C1B0C4D0C800CB30CE61D
:101ACC000D190D4B0D7E0DB10DE40E170E490E7C4C
:101ADC000EAF0EE20F150F470F7A0FAD0FE010137C
:101AEC001045107810AB10DE11111144117611A9AC
:101AFC0011DC120F1242127412A712DA130D1340DA
:101B0C00137213A513D8140B143E147014A314D60B
:101B1C001509153C156E15A115D41607163A166C39
:101B2C00169F16D217051738176A179D17D018036A
:101B3C0018361868189B18CE190119341967199999
:101B4C0019CC19FF1A321A651A971ACA1AFD1B30CA
:101B5C001B631B951BC81BFB1C2E1C611C931CC6FA
:101B6C001CF91D2C1D5F1D911DC41DF71E2A1E5D29
:101B7C001E8F1EC21EF51F281F5B1F8D1FC01FF35B
:101B8C0020262059208B20BE20F121242157218989
:101B9C0021BC21EF22222255228822BA22ED2320B9
:101BAC002353238623B823EB241E2451248424B6E8
:101BBC0024E9251C254F258225B425E7261A264D18
:101BCC00268026B226E52718274B277E27B027E349
:101BDC0028162849287C28AE28E129142947297A77
:101BEC0029AC29DF2A122A452A782AAB2ADD2B10A8
:101BFC002B432B762BA92BDB2C0E2C412C742CA7D6
:101C0C002CD92D0C2D3F2D722DA52DD72E0A2E3D06
:101C1C002E702EA32ED52F082F3B2F6E2FA12FD336
:101C2C0030063039306C309F30D131043137316A65
:101C3C00319D31CF320232353268329B32CE330095
:101C4C0033333366339933CC33FE343134643497C5
:101C5C0034CA34FC352F3562359535C835FA362DF6
:101C6C003660369336C636F8372B375E379137C425
:101C7C0037F63829385C388F38C238F43927395A56
:101C8C00398D39C039F23A253A583A8B3ABE3AF086
:101C9C003B233B563B893BBC3BEF3C213C543C87B4
:101CAC003CBA3CED3D1F3D523D853DB83DEB3E1DE4
:101CBC003E503E833EB63EE93F1B3F4E3F813FB414
:101CCC003FE74019404C407F40B240E54117414A44
:101CDC00417D41B041E342154248427B42AE42E174
:101CEC0043134346437943AC43DF441244444477A3
:101CFC0044AA44DD45104542457545A845DB460ED2
:101D0C004640467346A646D9470C473E477147A402
:101D1C0047D7480A483C486F48A248D54908493A31
:101D2C00496D49A049D34A064A384A6B4A9E4AD162
:101D3C004B044B364B694B9C4BCF4C024C354C6790
:101D4C004C9A4CCD4D004D334D654D984DCB4DFEC1
:101D5C004E314E634E964EC94EFC4F2F4F614F94F1
:101D6C004FC74FFA502D505F509250C550F8512B21
:101D7C00515D519051C351F65229525B528E52C152
:101D8C0052F453275359538C53BF53F25425545781
:101D9C00548A54BD54F055235556558855BB55EEB1
:101DAC0056215654568656B956EC571F57525784DF
:101DBC0057B757EA581D5850588258B558E8591B10
:101DCC00594E598059B359E65A195A4C5A7E5AB140
:101DDC005AE45B175B4A5B7C5BAF5BE25C155C486F
:101DEC005C7A5CAD5CE05D135D465D795DAB5DDEA0
:101DFC005E115E445E775EA95EDC5F0F5F425F75CD
:101E0C005FA75FDA600D6040607360A560D8610BFE
:101E1C00613E617161A361D66209623C626F62A12D
:101E2C0062D46307633A636D639F63D2640564385D
:101E3C00646B649D64D0650365366569659B65A7B5
:101E4C0065B265BD65C865D365DE65E965F465FF9A
:101E5C00660A66156620662B66366641664C6657C2
:101E6C006662666D66786683668E669966A466AFF2
:101E7C0066BA66C566D066DB66E666F166FC670820
:101E8C006713671E67296734673F674A6755676042
:101E9C00676B67766781678C679767A267AD67B872
:101EAC0067C367CE67D967E467EF67FA68056810A0
:101EBC00681B68266831683C68476852685D6868CA
:101ECC006874687F688A689568A068AB68B668C1F2
:101EDC0068CC68D768E268ED68F86903690E69191F
:101EEC006924692F693A69456950695B696669714A
:101EFC00697C69876992699D69A869B369BE69C97A
:101F0C0069D569E069EB69F66A016A0C6A176A229D
:101F1C006A2D6A386A436A4E6A596A646A6F6A7AC9
:101F2C006A856A906A9B6AA66AB16ABC6AC76AD2F9
:101F3C006ADD6AE86AF36AFE6B096B146B1F6B2A25
:101F4C006B356B416B4C6B576B626B6D6B786B834A
:101F5C006B8E6B996BA46BAF6BBA6BC56BD06BDB79
:101F6C006BE66BF16BFC6C076C126C1D6C286C33A4
:101F7C006C3E6C496C546C5F6C6A6C756C806C8BD1
:101F8C006C966CA26CAD6CB86CC36CCE6CD96CE4FA
:101F9C006CEF6CFA6D056D106D1B6D266D316D3C23
:101FAC006D476D526D5D6D686D736D7E6D896D9451
:101FBC006D9F6DAA6DB56DC06DCB6DD66DE16DEC81
:101FCC006DF76E026E0E6E196E246E2F6E3A6E45A4
:101FDC006E506E5B6E666E716E7C6E876E926E9DD1
:101FEC006EA86EB36EBE6EC96ED46EDF6EEA6EF501
:101FFC006F006F0B6F166F216F2C6F376F426F4D29
:10200C006F586F636F6E6F7A6F856F906F9B6FA653
:10201C006FB16FBC6FC76FD26FDD6FE86FF36FFE80
:10202C0070097014701F702A70357040704B7056A8
:10203C007061706C70777082708D709870A370AED8
:10204C0070B970C470CF70DB70E670F170FC710702
:10205C007112711D71287133713E71497154715F28
:10206C00716A71757180718B719671A171AC71B758
:10207C0071C271CD71D871E371EE71F97204720F86
:10208C00721A72257230723B72477252725D7268AC
:10209C007273727E72897294729F72AA72B572C0D8
:1020AC0072CB72D672E172EC72F77302730D731805
:1020BC007323732E73397344734F735A7365737030
:1020CC00737B73867391739C73A873B373BE73C95C
:1020DC0073D473DF73EA73F57400740B7416742184
:1020EC00742C74377442744D74587463746E7479B0
:1020FC007484748F749A74A574B074BB74C674D1E0
:10210C0074DC74E774F274FD75087514751F752A08
:10211C0075357540754B75567561756C757775822F
:10212C00758D759875A375AE75B975C475CF75DA5F
:10213C0075E575F075FB76067611761C762776328A
:10214C00763D76487653765E766976757680768BB4
:10215C00769676A176AC76B776C276CD76D876E3DF
:10216C0076EE76F97704770F771A77257730773B09
:10217C0077467751775C77677772777D7788779337
:10218C00779E77A977B477BF77CA77D577E177EC65
:10219C0077F77802780D78187823782E7839784488
:1021AC00784F785A78657870787B78867891789CB7
:1021BC0078A778B278BD78C878D378DE78E978F4E7
:1021CC0078FF790A79157920792B79367941794D0F
:1021DC0079587963796E79797984798F799A79A537
:1021EC0079B079BB79C679D179DC79E779F279FD67
:1021FC007A087A137A1E7A297A347A3F7A4A7A558F
:10220C007A607A6B7A767A817A8C7A977AA27AAEBD
:10221C007AB97AC47ACF7ADA7AE57AF07AFB7B06E5
:10222C007B117B1C7B277B327B3D7B487B537B5E0E
:10223C007B697B747B7F7B8A7B957BA07BAB7BB63E
:10224C007BC17BCC7BD77BE27BED7BF87C037C0E6C
:10225C007C1A7C257C307C3B7C467C517C5C7C678E
:10226C007C727C7D7C887C937C9E7CA97CB47CBFBE
:10227C007CCA7CD57CE07CEB7CF67D017D0C7D17EB
:10228C007D227D2D7D387D437D4E7D597D647D6F16
:10229C007D7B7D867D917D9C7DA77DB27DBD7DC83E
:1022AC007DD37DDE7DE97DF47DFF7E0A7E157E206B
:1022BC007E2B7E367E417E4C7E577E627E6D7E7896
:1022CC007E837E8E7E997EA47EAF7EBA7EC57ED0C6
:1022DC007EDB7EE77EF27EFD7F087F137F1E7F29EB
:1022EC007F347F3F7F4A7F557F607F6B7F767F8116
:1022FC007F8C7F977FA27FAD7FB87FC37FCE7FD946
:10230C007FE47FEF7FFA80058010801B8026803170
:10231C00803C80488053805E80698074807F808A96
:10232C00809580A080AB80B680C180CC80D780E2C5
:10233C0080ED80F88103810E81198124812F813AEF
:10234C0081458150815B81668171817C818781921D
:10235C00819D81A881B481BF81CA81D581E081EB47
:10236C0081F68201820C82178222822D823882436E
:10237C00824E82598264826F827A82858290829B9D
:10238C0082A682B182BC82C782D282DD82E882F3CD
:10239C0082FE830983148320832B83368341834CF1
:1023AC0083578362836D83788383838E839983A41D
:1023BC0083AF83BA83C583D083DB83E683F183FC4D
:1023CC0084078412841D84288433843E8449845475
:1023DC00845F846A84758481848C849784A284ADA0
:1023EC0084B884C384CE84D984E484EF84FA8505CC
:1023FC008510851B85268531853C85478552855DF5
:10240C0085688573857E85898594859F85AA85B524
:10241C0085C085CB85D685E185ED85F88603860E4E
:10242C0086198624862F863A86458650865B866674
:10243C008671867C86878692869D86A886B386BEA4
:10244C0086C986D486DF86EA86F58700870B8716D1
:10245C008721872C87378742874E87598764876FF8
:10246C00877A87858790879B87A687B187BC87C724
:10247C0087D287DD87E887F387FE88098814881F51
:10248C00882A88358840884B88568861886C88777C
:10249C008882888D889888A388AE88BA88C588D0A9
:1024AC0088DB88E688F188FC89078912891D8928D0
:1024BC008933893E89498954895F896A89758980FC
:1024CC00898B899689A189AC89B789C289CD89D82C
:1024DC0089E389EE89F98A048A0F8A1B8A268A3154
:1024EC008A3C8A478A528A5D8A688A738A7E8A897C
:1024FC008A948A9F8AAA8AB58AC08ACB8AD68AE1AC
:10250C008AEC8AF78B028B0D8B188B238B2E8B39D5
:10251C008B448B4F8B5A8B658B708B7B8B878B9201
:10252C008B9D8BA88BB38BBE8BC98BD48BDF8BEA2B
:10253C008BF58C008C0B8C168C218C2C8C378C4254
:10254C008C4D8C588C638C6E8C798C848C8F8C9A83
:10255C008CA58CB08CBB8CC68CD18CDC8CE78CF3B2
:10256C008CFE8D098D148D1F8D2A8D358D408D4BD4
:10257C008D568D618D6C8D778D828D8D8D988DA303
:10258C008DAE8DB98DC48DCF8DDA8DE58DF08DFB33
:10259C008E068E118E1C8E278E328E3D8E488E545A
:1025AC008E5F8E6A8E758E808E8B8E968EA18EAC83
:1025BC008EB78EC28ECD8ED88EE38EEE8EF98F04B2
:1025CC008F0F8F1A8F258F308F3B8F468F518F5CDB
:1025DC008F678F728F7D8F888F938F9E8FA98FB40B
:1025EC008FC08FCB8FD68FE18FEC8FF79002900D31
:1025FC0090189023902E90399044904F905A90655B
:10260C009070907B90869091909C90A790B290BD8A
:10261C0090C890D390DE90E990F490FF910A9115B8
:10262C009121912C91379142914D91589163916EDA
:10263C0091799184918F919A91A591B091BB91C60A
:10264C0091D191DC91E791F291FD92089213921E37
:10265C0092299234923F924A92559260926B927662
:10266C009281928D929892A392AE92B992C492CF8B
:10267C0092DA92E592F092FB93069311931C9327B6
:10268C009332933D93489353935E93699374937FE2
:10269C00938A939593A093AB93B693C193CC93D712
:1026AC0093E293EE93F99404940F941A9425943036
:1026BC00943B94469451945C94679472947D948862
:1026CC009493949E94A994B494BF94CA94D594E092
:1026DC0094EB94F69501950C95179522952D9538BC
:1026EC009543954E955A95659570957B95869591E4
:1026FC00959C95A795B295BD95C895D395DE95E912
:10270C0095F495FF960A96159620962B963696413B
:10271C00964C96579662966D96789683968E969969
:10272C0096A496AF96BA96C696D196DC96E796F294
:10273C0096FD97089713971E97299734973F974ABA
:10274C0097559760976B97769781978C979797A2E9
:10275C0097AD97B897C397CE97D997E497EF97FA19
:10276C0098059810981B98279832983D984898533C
:10277C00985E98699874987F988A989598A098AB69
:10278C0098B698C198CC98D798E298ED98F8990398
:10279C00990E99199924992F993A99459950995BC1
:1027AC0099669971997C99879993999E99A999B4ED
:1027BC0099BF99CA99D599E099EB99F69A019A0C17
:1027CC009A179A229A2D9A389A439A4E9A599A6441
:1027DC009A6F9A7A9A859A909A9B9AA69AB19ABC71
:1027EC009AC79AD29ADD9AE89AF49AFF9B0A9B159B
:1027FC009B209B2B9B369B419B4C9B579B629B6DC1
:10280C009B789B839B8E9B999BA49BAF9BBA9BC5F0
:10281C009BD09BDB9BE69BF19BFC9C079C129C1D1D
:10282C009C289C339C3E9C499C549C609C6B9C7645
:10283C009C819C8C9C979CA29CAD9CB89CC39CCE70
:10284C009CD99CE49CEF9CFA9D059D109D1B9D269C
:10285C009D319D3C9D479D529D5D9D689D739D7EC8
:10286C009D899D949D9F9DAA9DB59DC19DCC9DD7F5
:10287C009DE29DED9DF89E039E0E9E199E249E2F1B
:10288C009E3A9E459E509E5B9E669E719E7C9E8748
:10289C009E929E9D9EA89EB39EBE9EC99ED49EDF78
:1028AC009EEA9EF59F009F0B9F169F219F2D9F38A0
:1028BC009F439F4E9F599F649F6F9F7A9F859F90C8
:1028CC009F9B9FA69FB19FBC9FC79FD29FDD9FE8F8
:1028DC009FF39FFEA009A014A01FA02AA035A04022
:1028EC00A04BA056A061A06CA077A082A08DA0994F
:1028FC00A0A4A0AFA0BAA0C5A0D0A0DBA0E6A0F178
:10290C00A0FCA107A112A11DA128A133A13EA149A0
:10291C00A154A15FA16AA175A180A18BA196A1A1CF
:10292C00A1ACA1B7A1C2A1CDA1D8A1E3A1EEA1FAFE
:10293C00A205A210A21BA226A231A23CA247A2521F
:10294C00A25DA268A273A27EA289A294A29FA2AA4F
:10295C00A2B5A2C0A2CBA2D6A2E1A2ECA2F7A3027E
:10296C00A30DA318A323A32EA339A344A34FA35AA7
:10297C00A366A371A37CA387A392A39DA3A8A3B3CF
:10298C00A3BEA3C9A3D4A3DFA3EAA3F5A400A40BFD
:10299C00A416A421A42CA437A442A44DA458A46327
:1029AC00A46EA479A484A48FA49AA4A5A4B0A4BB57
:1029BC00A4C7A4D2A4DDA4E8A4F3A4FEA509A5147D
:1029CC00A51FA52AA535A540A54BA556A561A56CA7
:1029DC00A577A582A58DA598A5A3A5AEA5B9A5C4D7
:1029EC00A5CFA5DAA5E5A5F0A5FBA606A611A61C04
:1029FC00A627A633A63EA649A654A65FA66AA67528
:102A0C00A680A68BA696A6A1A6ACA6B7A6C2A6CD56
:102A1C00A6D8A6E3A6EEA6F9A704A70FA71AA72582
:102A2C00A730A73BA746A751A75CA767A772A77DAE
:102A3C00A788A794A79FA7AAA7B5A7C0A7CBA7D6D7
:102A4C00A7E1A7ECA7F7A802A80DA818A823A82E01
:102A5C00A839A844A84FA85AA865A870A87BA8862E
:102A6C00A891A89CA8A7A8B2A8BDA8C8A8D3A8DE5E
:102A7C00A8E9A8F4A900A90BA916A921A92CA93782
:102A8C00A942A94DA958A963A96EA979A984A98FAE
:102A9C00A99AA9A5A9B0A9BBA9C6A9D1A9DCA9E7DE
:102AAC00A9F2A9FDAA08AA13AA1EAA29AA34AA3F08
:102ABC00AA4AAA55AA60AA6CAA77AA82AA8DAA9831
:102ACC00AAA3AAAEAAB9AAC4AACFAADAAAE5AAF05E
:102ADC00AAFBAB06AB11AB1CAB27AB32AB3DAB4887
:102AEC00AB53AB5EAB69AB74AB7FAB8AAB95ABA0B6
:102AFC00ABABABB6ABC1ABCDABD8ABE3ABEEABF9E1
:102B0C00AC04AC0FAC1AAC25AC30AC3BAC46AC5105
:102B1C00AC5CAC67AC72AC7DAC88AC93AC9EACA935
:102B2C00ACB4ACBFACCAACD5ACE0ACEBACF6AD0164
:102B3C00AD0CAD17AD22AD2DAD39AD44AD4FAD5A89
:102B4C00AD65AD70AD7BAD86AD91AD9CADA7ADB2B5
:102B5C00ADBDADC8ADD3ADDEADE9ADF4ADFFAE0AE4
:102B6C00AE15AE20AE2BAE36AE41AE4CAE57AE620D
:102B7C00AE6DAE78AE83AE8EAE9AAEA5AEB0AEBB39
:102B8C00AEC6AED1AEDCAEE7AEF2AEFDAF08AF1363
:102B9C00AF1EAF29AF34AF3FAF4AAF55AF60AF6B8D
:102BAC00AF76AF81AF8CAF97AFA2AFADAFB8AFC3BD
:102BBC00AFCEAFD9AFE4AFEFAFFAB006B011B01CE7
:102BCC00B027B032B03DB048B053B05EB069B0740D
:102BDC00B07FB08AB095B0A0B0ABB0B6B0C1B0CC3D
:102BEC00B0D7B0E2B0EDB0F8B103B10EB119B12469
:102BFC00B12FB13AB145B150B15BB167B172B17D92
:102C0C00B188B193B19EB1A9B1B4B1BFB1CAB1D5BC
:102C1C00B1E0B1EBB1F6B201B20CB217B222B22DE7
:102C2C00B238B243B24EB259B264B26FB27AB28514
:102C3C00B290B29BB2A6B2B1B2BCB2C7B2D3B2DE42
:102C4C00B2E9B2F4B2FFB30AB315B320B32BB33667
:102C5C00B341B34CB357B362B36DB378B383B38E94
:102C6C00B399B3A4B3AFB3BAB3C5B3D0B3DBB3E6C4
:102C7C00B3F1B3FCB407B412B41DB428B433B43FED
:102C8C00B44AB455B460B46BB476B481B48CB49714
:102C9C00B4A2B4ADB4B8B4C3B4CEB4D9B4E4B4EF44
:102CAC00B4FAB505B510B51BB526B531B53CB5476D
:102CBC00B552B55DB568B573B57EB589B594B5A09B
:102CCC00B5ABB5B6B5C1B5CCB5D7B5E2B5EDB5F8C4
:102CDC00B603B60EB619B624B62FB63AB645B650EC
:102CEC00B65BB666B671B67CB687B692B69DB6A81C
:102CFC00B6B3B6BEB6C9B6D4B6DFB6EAB6F5B7004B
:102D0C00B70CB717B722B72DB738B743B74EB7596B
:102D1C00B764B76FB77AB785B790B79BB7A6B7B19B
:102D2C00B7BCB7C7B7D2B7DDB7E8B7F3B7FEB809CA
:102D3C00B814B81FB82AB835B840B84BB856B861F3
:102D4C00B86DB878B883B88EB899B8A4B8AFB8BA1B
:102D5C00B8C5B8D0B8DBB8E6B8F1B8FCB907B91249
:102D6C00B91DB928B933B93EB949B954B95FB96A73
:102D7C00B975B980B98BB996B9A1B9ACB9B7B9C2A3
:102D8C00B9CDB9D9B9E4B9EFB9FABA05BA10BA1BC9
:102D9C00BA26BA31BA3CBA47BA52BA5DBA68BA73F3
:102DAC00BA7EBA89BA94BA9FBAAABAB5BAC0BACB23
:102DBC00BAD6BAE1BAECBAF7BB02BB0DBB18BB234F
:102DCC00BB2EBB3ABB45BB50BB5BBB66BB71BB7C74
:102DDC00BB87BB92BB9DBBA8BBB3BBBEBBC9BBD4A3
:102DEC00BBDFBBEABBF5BC00BC0BBC16BC21BC2CCE
:102DFC00BC37BC42BC4DBC58BC63BC6EBC79BC84FB
:102E0C00BC8FBC9ABCA6BCB1BCBCBCC7BCD2BCDD24
:102E1C00BCE8BCF3BCFEBD09BD14BD1FBD2ABD354D
:102E2C00BD40BD4BBD56BD61BD6CBD77BD82BD8D7A
:102E3C00BD98BDA3BDAEBDB9BDC4BDCFBDDABDE5AA
:102E4C00BDF0BDFBBE06BE12BE1DBE28BE33BE3ECF
:102E5C00BE49BE54BE5FBE6ABE75BE80BE8BBE96FA
:102E6C00BEA1BEACBEB7BEC2BECDBED8BEE3BEEE2A
:102E7C00BEF9BF04BF0FBF1ABF25BF30BF3BBF4653
:102E8C00BF51BF5CBF67BF73BF7EBF89BF94BF9F7D
:102E9C00BFAABFB5BFC0BFCBBFD6BFE1BFECBFF7AA
:102EAC00C002C00DC018C023C02EC039C044C04FD2
:102EBC00C05AC065C070C07BC086C091C09CC0A702
:102ECC00C0B2C0BDC0C8C0D3C0DFC0EAC0F5C1002D
:102EDC00C10BC116C121C12CC137C142C14DC15852
:102EEC00C163C16EC179C184C18FC19AC1A5C1B082
:102EFC00C1BBC1C6C1D1C1DCC1E7C1F2C1FDC208B1
:102F0C00C213C21EC229C234C240C24BC256C261D5
:102F1C00C26CC277C282C28DC298C2A3C2AEC2B901
:102F2C00C2C4C2CFC2DAC2E5C2F0C2FBC306C3112F
:102F3C00C31CC327C332C33DC348C353C35EC36959
:102F4C00C374C37FC38AC395C3A0C3ACC3B7C3C286
:102F5C00C3CDC3D8C3E3C3EEC3F9C404C40FC41AAE
:102F6C00C425C430C43BC446C451C45CC467C472D9
:102F7C00C47DC488C493C49EC4A9C4B4C4BFC4CA09
:102F8C00C4D5C4E0C4EBC4F6C501C50DC518C52332
:102F9C00C52EC539C544C54FC55AC565C570C57B59
:102FAC00C586C591C59CC5A7C5B2C5BDC5C8C5D389
:102FBC00C5DEC5E9C5F4C5FFC60AC615C620C62BB5
:102FCC00C636C641C64CC657C662C66DC679C684DF
:102FDC00C68FC69AC6A5C6B0C6BBC6C6C6D1C6DC09
:102FEC00C6E7C6F2C6FDC708C713C71EC729C73434
:102FFC00C73FC74AC755C760C76BC776C781C78C61
:10300C00C797C7A2C7ADC7B8C7C3C7CEC7D9C7E58F
:10301C00C7F0C7FBC806C811C81CC827C832C83DB2
:10302C00C848C853C85EC869C874C87FC88AC895E0
:10303C00C8A0C8ABC8B6C8C1C8CCC8D7C8E2C8ED10
:10304C00C8F8C903C90EC919C924C92FC93AC94638
:10305C00C951C95CC967C972C97DC988C993C99E60
:10306C00C9A9C9B4C9BFC9CAC9D5C9E0C9EBC9F690
:10307C00CA01CA0CCA17CA22CA2DCA38CA43CA4EB8
:10308C00CA59CA64CA6FCA7ACA85CA90CA9BCAA6E8
:10309C00CAB2CABDCAC8CAD3CADECAE9CAF4CAFF10
:1030AC00CB0ACB15CB20CB2BCB36CB41CB4CCB5738
:1030BC00CB62CB6DCB78CB83CB8ECB99CBA4CBAF68
:1030CC00CBBACBC5CBD0CBDBCBE6CBF1CBFCCC0797
:1030DC00CC13CC1ECC29CC34CC3FCC4ACC55CC60B8
:1030EC00CC6BCC76CC81CC8CCC97CCA2CCADCCB8E8
:1030FC00CCC3CCCECCD9CCE4CCEFCCFACD05CD1016
:10310C00CD1BCD26CD31CD3CCD47CD52CD5DCD683F
:10311C00CD73CD7FCD8ACD95CDA0CDABCDB6CDC168
:10312C00CDCCCDD7CDE2CDEDCDF8CE03CE0ECE1994
:10313C00CE24CE2FCE3ACE45CE50CE5BCE66CE71BF
:10314C00CE7CCE87CE92CE9DCEA8CEB3CEBECEC9EF
:10315C00CED4CEE0CEEBCEF6CF01CF0CCF17CF2214
:10316C00CF2DCF38CF43CF4ECF59CF64CF6FCF7A3F
:10317C00CF85CF90CF9BCFA6CFB1CFBCCFC7CFD26F
:10318C00CFDDCFE8CFF3CFFED009D014D01FD02A9B
:10319C00D035D040D04CD057D062D06DD078D083C1
:1031AC00D08ED099D0A4D0AFD0BAD0C5D0D0D0DBEF
:1031BC00D0E6D0F1D0FCD107D112D11DD128D1331A
:1031CC00D13ED149D154D15FD16AD175D180D18B47
:1031DC00D196D1A1D1ACD1B8D1C3D1CED1D9D1E472
:1031EC00D1EFD1FAD205D210D21BD226D231D23C99
:1031FC00D247D252D25DD268D273D27ED289D294C7
:10320C00D29FD2AAD2B5D2C0D2CBD2D6D2E1D2ECF6
:10321C00D2F7D302D30DD319D324D32FD33AD3451A
:10322C00D350D35BD366D371D37CD387D392D39D46
:10323C00D3A8D3B3D3BED3C9D3D4D3DFD3EAD3F576
:10324C00D400D40BD416D421D42CD437D442D44D9E
:10325C00D458D463D46ED479D485D490D49BD4A6CA
:10326C00D4B1D4BCD4C7D4D2D4DDD4E8D4F3D4FEF6
:10327C00D509D514D51FD52AD535D540D54BD5561E
:10328C00D561D56CD577D582D58DD598D5A3D5AE4E
:10329C00D5B9D5C4D5CFD5DAD5E6D5F1D5FCD60779
:1032AC00D612D61DD628D633D63ED649D654D65F9E
:1032BC00D66AD675D680D68BD696D6A1D6ACD6B7CE
:1032CC00D6C2D6CDD6D8D6E3D6EED6F9D704D70FFC
:1032DC00D71AD725D730D73BD746D752D75DD76823
:1032EC00D773D77ED789D794D79FD7AAD7B5D7C04E
:1032FC00D7CBD7D6D7E1D7ECD7F7D802D80DD8187B
:10330C00D823D82ED839D844D84FD85AD865D870A5
:10331C00D87BD886D891D89CD8A7D8B3D8BED8C9D2
:10332C00D8D4D8DFD8EAD8F5D900D90BD916D921F9
:10333C00D92CD937D942D94DD958D963D96ED97925
:10334C00D984D98FD99AD9A5D9B0D9BBD9C6D9D155
:10335C00D9DCD9E7D9F2D9FDDA08DA13DA1FDA2A7F
:10336C00DA35DA40DA4BDA56DA61DA6CDA77DA82A5
:10337C00DA8DDA98DAA3DAAEDAB9DAC4DACFDADAD5
:10338C00DAE5DAF0DAFBDB06DB11DB1CDB27DB3200
:10339C00DB3DDB48DB53DB5EDB69DB74DB7FDB8B2C
:1033AC00DB96DBA1DBACDBB7DBC2DBCDDBD8DBE355
:1033BC00DBEEDBF9DC04DC0FDC1ADC25DC30DC3B7F
:1033CC00DC46DC51DC5CDC67DC72DC7DDC88DC93AD
:1033DC00DC9EDCA9DCB4DCBFDCCADCD5DCE0DCECDC
:1033EC00DCF7DD02DD0DDD18DD23DD2EDD39DD44FE
:1033FC00DD4FDD5ADD65DD70DD7BDD86DD91DD9C2D
:10340C00DDA7DDB2DDBDDDC8DDD3DDDEDDE9DDF45C
:10341C00DDFFDE0ADE15DE20DE2BDE36DE41DE4C85
:10342C00DE58DE63DE6EDE79DE84DE8FDE9ADEA5AC
:10343C00DEB0DEBBDEC6DED1DEDCDEE7DEF2DEFDDC
:10344C00DF08DF13DF1EDF29DF34DF3FDF4ADF5504
:10345C00DF60DF6BDF76DF81DF8CDF97DFA2DFAD34
:10346C00DFB9DFC4DFCFDFDADFE5DFF0DFFBE0065B
:10347C00E011E01CE027E032E03DE048E053E05E84
:10348C00E069E074E07FE08AE095E0A0E0ABE0B6B4
:10349C00E0C1E0CCE0D7E0E2E0EDE0F8E103E10EE2
:1034AC00E119E125E130E13BE146E151E15CE16705
:1034BC00E172E17DE188E193E19EE1A9E1B4E1BF34
:1034CC00E1CAE1D5E1E0E1EBE1F6E201E20CE21761
:1034DC00E222E22DE238E243E24EE259E264E26F8C
:1034EC00E27AE286E291E29CE2A7E2B2E2BDE2C8B5
:1034FC00E2D3E2DEE2E9E2F4E2FFE30AE315E320E1
:10350C00E32BE336E341E34CE357E362E36DE3780B
:10351C00E383E38EE399E3A4E3AFE3BAE3C5E3D03B
:10352C00E3DBE3E6E3F2E3FDE408E413E41EE42961
:10353C00E434E43FE44AE455E460E46BE476E4818B
:10354C00E48CE497E4A2E4ADE4B8E4C3E4CEE4D9BB
:10355C00E4E4E4EFE4FAE505E510E51BE526E531E6
:10356C00E53CE547E552E55EE569E574E57FE58A0E
:10357C00E595E5A0E5ABE5B6E5C1E5CCE5D7E5E23B
:10358C00E5EDE5F8E603E60EE619E624E62FE63A65
:10359C00E645E650E65BE666E671E67CE687E69293
:1035AC00E69DE6A8E6B3E6BFE6CAE6D5E6E0E6EBBE
:1035BC00E6F6E701E70CE717E722E72DE738E743E4
:1035CC00E74EE759E764E76FE77AE785E790E79B13
:1035DC00E7A6E7B1E7BCE7C7E7D2E7DDE7E8E7F343
:1035EC00E7FEE809E814E81FE82BE836E841E84C68
:1035FC00E857E862E86DE878E883E88EE899E8A493
:10360C00E8AFE8BAE8C5E8D0E8DBE8E6E8F1E8FCC2
:10361C00E907E912E91DE928E933E93EE949E954EA
:10362C00E95FE96AE975E980E98CE997E9A2E9AD16
:10363C00E9B8E9C3E9CEE9D9E9E4E9EFE9FAEA0541
:10364C00EA10EA1BEA26EA31EA3CEA47EA52EA5D6A
:10365C00EA68EA73EA7EEA89EA94EA9FEAAAEAB59A
:10366C00EAC0EACBEAD6EAE1EAECEAF8EB03EB0EC5
:10367C00EB19EB24EB2FEB3AEB45EB50EB5BEB66EA
:10368C00EB71EB7CEB87EB92EB9DEBA8EBB3EBBE1A
:10369C00EBC9EBD4EBDFEBEAEBF5EC00EC0BEC1647
:1036AC00EC21EC2CEC37EC42EC4DEC59EC64EC6F6F
:1036BC00EC7AEC85EC90EC9BECA6ECB1ECBCECC79A
:1036CC00ECD2ECDDECE8ECF3ECFEED09ED14ED1FC7
:1036DC00ED2AED35ED40ED4BED56ED61ED6CED77F2
:1036EC00ED82ED8DED98EDA3EDAEEDB9EDC5EDD020
:1036FC00EDDBEDE6EDF1EDFCEE07EE12EE1DEE2846
:10370C00EE33EE3EEE49EE54EE5FEE6AEE75EE8071
:10371C00EE8BEE96EEA1EEACEEB7EEC2EECDEED8A1
:10372C00EEE3EEEEEEF9EF04EF0FEF1AEF25EF31CB
:10373C00EF3CEF47EF52EF5DEF68EF73EF7EEF89F1
:10374C00EF94EF9FEFAAEFB5EFC0EFCBEFD6EFE121
:10375C00EFECEFF7F002F00DF018F023F02EF0394B
:10376C00F044F04FF05AF065F070F07BF086F09278
:10377C00F09DF0A8F0B3F0BEF0C9F0D4F0DFF0EAA1
:10378C00F0F5F100F10BF116F121F12CF137F142CA
:10379C00F14DF158F163F16EF179F184F18FF19AF9
:1037AC00F1A5F1B0F1BBF1C6F1D1F1DCF1E7F1F229
:1037BC00F1FEF209F214F21FF22AF235F240F24B4A
:1037CC00F256F261F26CF277F282F28DF298F2A379
:1037DC00F2AEF2B9F2C4F2CFF2DAF2E5F2F0F2FBA9
:1037EC00F306F311F31CF327F332F33DF348F353D1
:1037FC00F35FF36AF375F380F38BF396F3A1F3ACF9
:10380C00F3B7F3C2F3CDF3D8F3E3F3EEF3F9F40427
:10381C00F40FF41AF425F430F43BF446F451F45C50
:10382C00F467F472F47DF488F493F49EF4A9F4B480
:10383C00F4BFF4CBF4D6F4E1F4ECF4F7F502F50DA7
:10384C00F518F523F52EF539F544F54FF55AF565D0
:10385C00F570F57BF586F591F59CF5A7F5B2F5BD00
:10386C00F5C8F5D3F5DEF5E9F5F4F5FFF60AF6152E
:10387C00F620F62BF637F642F64DF658F663F66E52
:10388C00F679F684F68FF69AF6A5F6B0F6BBF6C680
:10389C00F6D1F6DCF6E7F6F2F6FDF708F713F71EAD
:1038AC00F729F734F73FF74AF755F760F76BF776D8
:1038BC00F781F78CF798F7A3F7AEF7B9F7C4F7CF02
:1038CC00F7DAF7E5F7F0F7FBF806F811F81CF8272C
:1038DC00F832F83DF848F853F85EF869F874F87F58
:1038EC00F88AF895F8A0F8ABF8B6F8C1F8CCF8D788
:1038FC00F8E2F8EDF8F8F904F90FF91AF925F930AE
:10390C00F93BF946F951F95CF967F972F97DF988D7
:10391C00F993F99EF9A9F9B4F9BFF9CAF9D5F9E007
:10392C00F9EBF9F6FA01FA0CFA17FA22FA2DFA3831
:10393C00FA43FA4EFA59FA65FA70FA7BFA86FA915A
:10394C00FA9CFAA7FAB2FABDFAC8FAD3FADEFAE987
:10395C00FAF4FAFFFB0AFB15FB20FB2BFB36FB41B1
:10396C00FB4CFB57FB62FB6DFB78FB83FB8EFB99DF
:10397C00FBA4FBAFFBBAFBC5FBD1FBDCFBE7FBF20B
:10398C00FBFDFC08FC13FC1EFC29FC34FC3FFC4A30
:10399C00FC55FC60FC6BFC76FC81FC8CFC97FCA25F
:1039AC00FCADFCB8FCC3FCCEFCD9FCE4FCEFFCFA8F
:1039BC00FD05FD10FD1BFD26FD32FD3DFD48FD53B3
:1039CC00FD5EFD69FD74FD7FFD8AFD95FDA0FDABDF
:1039DC00FDB6FDC1FDCCFDD7FDE2FDEDFDF8FE030E
:1039EC00FE0EFE19FE24FE2FFE3AFE45FE50FE5B37
:1039FC00FE66FE71FE7CFE87FE92FE9EFEA9FEB464
:103A0C00FEBFFECAFED5FEE0FEEBFEF6FF01FF0C8C
:103A1C00FF17FF22FF2DFF38FF43FF4EFF59FF64B6
:103A2C00FF6FFF7AFF85FF90FF9BFFA6FFB1FFBCE6
:103A3C00FFC7FFD2FFDDFFE8FFF3FFFE303132336B
:043A4C0034353637A0
:100C9A0041004700C10441004800680000630000A9
:100CAA000001000100020002000300040004000524
:100CBA0000050006000600070008000800090009F0
:100CCA00000A000B000B000C000C000D000D000EBA
:100CDA00000F000F00100010001100120012001384
:100CEA00001300140015001500160016001700174F
:100CFA00001800190019001A001A001B001C001C19
:100D0A00001D001D001E001E001F002000200021E3
:100D1A0000210022002300230024002400250026AD
:100D2A00002600270027002800280029002A002A78
:100D3A00002B002B002C002D002D002E002E002F42
:100D4A00002F00300031003100320032003300340D
:100D5A0000340035003500360036003700380038D8
:100D6A0000390039003A003B003B003C003C003DA2
:100D7A00003E003E003F003F00400040004100426C
:100D8A000042004300430044004500450046004637
:100D9A0000470047004800490049004A004A004B02
:100DAA00004C004C004D004D004E004F004F0050CB
:100DBA000050005100510052005300530054005497
:100DCA000055005600560057005700580058005961
:100DDA00005A005A005B005B005C005D005D005E2B
:100DEA00005E005F006000600061006100620062F6
:100DFA0000630064006400650065006600670067C0
:100E0A000068006800690069006A006B006B006C8A
:100E1A00006C006D006E006E006F006F0070007154
:100E2A00007100720072007300730074007500751F
:100E3A000076007600770078007800790079007AE9
:100E4A00007A007B007C007C007D007D007E007FB4
:100E5A00007F00800080008100810082008300837F
:100E6A000084008400850086008600870087008849
:100E7A0000890089008A008A008B008B008C008D13
:100E8A00008D008E008E008F0090009000910091DE
:100E9A0000920092009300940094009500950096A9
:100EAA0000970097009800980099009A009A009B72
:100EBA00009B009C009C009D009E009E009F009F3E
:100ECA0000A000A100A100A200A200A300A300A408
:100EDA0000A500A500A600A600A700A800A800A9D2
:100EEA0000A900AA00AB00AB00AC00AC00AD00AD9D
:100EFA0000AE00AF00AF00B000B000B100B200B267
:100F0A0000B300B300B400B400B500B600B600B731
:100F1A0000B700B800B900B900BA00BA00BB00BCFB
:100F2A0000BC00BD00BD00BE00BE00BF00C000C0C6
:100F3A0000C100C100C200C300C300C400C400C590
:100F4A0000C500C600C700C700C800C800C900CA5B
:100F5A0000CA00CB00CB00CC00CC00CD00CE00CE26
:100F6A0000CF00CF00D000D100D100D200D200D3F0
:100F7A0000D400D400D500D500D600D600D700D8BA
:100F8A0000D800D900D900DA00DB00DB00DC00DC85
:100F9A0000DD00DD00DE00DF00DF00E000E000E150
:100FAA0000E200E200E300E300E400E500E500E619
:100FBA0000E600E700E700E800E900E900EA00EAE5
:100FCA0000EB00EC00EC00ED00ED00EE00EE00EFAF
:100FDA0000F000F000F100F100F200F300F300F479
:100FEA0000F400F500F600F600F700F700F800F844
:100FFA0000F900FA00FA00FB00FB00FC00FD00FD0E
:10100A0000FE00FE00FF00FF0100010101010102D4
:10101A00010201030104010401050105010601079A
:10102A0001070108010801090109010A010B010B65
:10103A00010C010C010D010E010E010F010F01102F
:10104A0001100111011201120113011301140115FA
:10105A0001150116011601170117011801190119C5
:10106A00011A011A011B011C011C011D011D011E8F
:10107A00011F011F01200120012101210122012359
:10108A000123012401240125012601260127012724
:10109A00012801280129012A012A012B012B012CEF
:1010AA00012D012E013001310132013301340135A4
:1010BA00013701380139013A013B013C013E013F48
:1010CA0001400141014201430145014601470148EE
:1010DA000149014A014C014D014E014F0150015293
:1010EA00015301540155015601570159015A015B37
:1010FA00015C015D015E01600161016201630164DD
:10110A000165016701680169016A016B016C016E81
:10111A00016F017001710172017301750176017726
:10112A0001780179017B017C017D017E017F0180CB
:10113A000182018301840185018601870189018A6F
:10114A00018B018C018D018E019001910192019315
:10115A0001940195019701980199019A019B019DBA
:10116A00019E019F01A001A101A201A401A501A65E
:10117A0001A701A801A901AB01AC01AD01AE01AF04
:10118A0001B001B201B301B401B501B601B701B9A9
:10119A0001BA01BB01BC01BD01BE01C001C101C24E
:1011AA0001C301C401C601C701C801C901CA01CBF3
:1011BA0001CD01CE01CF01D001D101D201D401D597
:1011CA0001D601D701D801D901DB01DC01DD01DE3D
:1011DA0001DF01E001E201E301E401E501E601E8E2
:1011EA0001E901EA01EB01EC01ED01EF01F001F186
:1011FA0001F201F301F401F601F701F801F901FA2C
:10120A0001FB01FD01FE01FF0200020102020204CC
:10121A0002050206020702080209020B020C020D6D
:10122A00020E020F02110212021302140215021612
:10123A0002180219021A021B021C021D021F0220B6
:10124A00022102220223022402260227022802295C
:10125A00022A022B022D022E022F02300231023301
:10126A0002340235023602370238023A023B023CA5
:10127A00023D023E023F024102420243024402454B
:10128A00024602480249024A024B024C024D024FF0
:10129A000250025102520253025402560257025A93
:1012AA00025C025F0261026302660268026A026D00
:1012BA00026F0272027402760279027B027D028058
:1012CA000282028402870289028B028E02900292B3
:1012DA00029502970299029C029E02A102A302A50C
:1012EA0002A802AA02AC02AF02B102B302B602B865
:1012FA0002BA02BD02BF02C102C402C602C902CBBF
:10130A0002CD02D002D202D402D702D902DB02DE17
:10131A0002E002E202E502E702E902EC02EE02F171
:10132A0002F302F502F802FA02FC02FF03010303C8
:10133A0003060308030A030D030F0311031403161C
:10134A000318031B031D0320032203240327032975
:10135A00032B032E03300332033503370339033CCF
:10136A00033E0340034303450348034A034C034F28
:10137A000351035303560358035A035D035F036182
:10138A00036403660368036B036D036F03720374DC
:10139A0003770379037B037E038003820385038734
:1013AA00038C03900395039A039F03A303A803AD39
:1013BA0003B103B603BB03BF03C403C903CE03D2FD
:1013CA0003D703DC03E003E503EA03EE03F303F8C0
:1013DA0003FD04010406040B040F04140419041E7B
:1013EA0004220427042C04300435043A043E04433E
:1013FA000448044D04510456045B045F0464046900
:10140A00046D04720477047C04800485048A048EC3
:10141A0004930498049C04A104A604AB04AF04B486
:10142A0004BD04C704D004DA04E304EC04F604FFA0
:10143A0005090512051B0525052E05380541054B2D
:10144A000554055D05670570057A0583058C0596C3
:10145A00059F05A905B205BB05C505CE05D805E159
:10146A000734088609D90B2B0C7E0DD00F23107573
:10147A0011C8131A146D15C01712186519B71B0A6B
:10148A001C5C1DAF1F01205421A722F9244C259E64
:10149A0026F1284329962AE82C3B2D8D2EE0410877
:1014AA006300410864004208650000410867004182
:1014BA0000000041000101410868004200020000EA
:1014CA0042000400004200060000420008000042F8
:1014DA00000A000042000C00004108690041086A45
:0A14EA008041086B8042086C00008E
:105A4D00900CFAE0FEA3E0FF900CF6E0FCA3E0FD65
:105A5D00B50719ECB50615900CF8E0FEA3E0FFEDC7
:0E5A6D00B50709ECB5060520C502D322C322F9
:105BBF00E4F584758810758902758E02758A0175F2
:065BCF008C0143A8022234
:035C3C00025941C9
:0D5BFF00E4F584759A4075F809759D302213
:1019E600E4F58475E880900863E0F5BB75840275BC
:1019F600BCF975E880A3E0F5BBE4F58443E7122261
:075C2500E4F58475D10222B1
:105B8D0075840FE4F5AD75A4CF75A50175A67F7568
:095B9D00A77F75E10375E34022C6
:10581E00E4FFFE75840F438A0353A1DFF58475B749
:10582E003075840F43A120438901758D01758F0159
:10583E00758E040FBF00010EEF640F4E70F5438995
:10584E0002E58920E4130FBF00010EBE0FF3BFFF68
:0C585E00F0E4F58443EF1080E875970239
:01586A00221B
:101A1B0012581E125B8D125BBF125BFF125C2512FC
:051A2B0019E6025C3C1D
:104E7C0075FFDE75FFAD9000467450F0121A1BD210
:104E8C00AF125BA602501AAF84E4F584900C70E06C
:104E9C0004F08F84900048E06008121A33E490000C
:104EAC0048F0125A1DEF60DF900D44E0FFB40B0286
:104EBC00D204EF64317044900046E0FF900D45E061
:104ECC006F7038125A4D50FB900046E0FF125BEAAF
:104EDC00125A4D50FB900D46E0FFA3E0FDA3E0FB02
:104EEC00A3E0900C74F0125038125A4D50FB900005
:104EFC0046E0FF125BD5125A4D50FB900D44E06416
:104F0C0032703E900046E0FF900D45E06F7032121B
:104F1C005A4D50FB900046E0FF125BEA125A4D507E
:104F2C00FB900D46E0FFA3E0FDA3E0FB12188612F8
:104F3C005A4D50FB900046E0FF125BD5125A4D5073
:104F4C00FB900D44E0642D703E900046E0FF900D08
:104F5C0045E06F7032125A4D50FB900046E0FF1244
:104F6C005BEA125A4D50FB900D46E0FFA3E0FDA307
:104F7C00E0FB1252D4125A4D50FB900046E0FF1247
:104F8C005BD5125A4D50FB900D44E0642E703E9050
:104F9C000046E0FF900D45E06F7032125A4D50FB09
:104FAC00900046E0FF125BEA125A4D50FB900D4602
:104FBC00E0FFA3E0FDA3E0FB1251E8125A4D50FBB9
:104FCC00900046E0FF125BD5125A4D50FB900D44F9
:104FDC00E0FFB414089000477401F0C205EFB4155B
:104FEC0005E4900047F0900047E07003024E939068
:104FFC000D44E014601E046003024E93900D45E0D6
:10500C00FFC3941E4003024E93900D12EFF0125A00
:10501C00F4024E93900D45E0FFC3941E4003024EE4
:0C502C0093900D12EFF0121A33024E9315
:031A0600023A5051
:103A5000C0E0C0F0C083C082C0D075D000C000C03C
:0D3A600001C002C003C004C005C006C007BD
:103A6D00900CA6740FF0A374FFF0A37408F0A37468
:103A7D0020F0900867E014600F1460111460392471
:103A8D00037038125C388033125C0C802E90086500
:103A9D00E4F0A3F0124A40900866E004F07006903E
:103AAD000865E004F0C3900866E09408900865E0AE
:103ABD006480948040DE8003125B54900867E004BC
:103ACD00F0C3648094844002E4F0900CA8E0FEA35F
:103ADD00E0FBAA06E4F9F8900CA6E0FEA3E0FFE4F3
:103AED00FCFD1216A2900CA21217E6900867E0FFDB
:0E3AFD0075F002121612AFF0EF700302420CC9
:073B0B00900CACE4F0A3F004
:103B1200900CADE025E0FF900CACE033FE743C2F3E
:103B2200F9741A3EFA900CCA74FFF0A3EAF0A3E902
:103B3200F0900CCAE0FBA3E0FAA3E0F9121634FD00
:103B4200540FFB900CCDE4F0A3EBF0EDC4540FFD49
:103B5200A3E4F0A3EDF0900CCAE0FB900001121672
:103B62004D540FFD900CD1E4F0A3EDF074132FF53A
:103B720082740D3EF583E0FEA3E0FFE4FCFD900CB1
:103B8200D31217E6900CACE0FEA3E0FF4E6006EF06
:103B920064054E7016900CCEE025E0FF900CCDE04F
:103BA20033FE74262FF58274008014900CADE0254C
:103BB200E0FF900CACE033FE741D2FF582740D3ED5
:103BC200F583E0FEA3E0FFE4FCFD900CC21217E6D1
:103BD200900CC2E0F8A3E0F9A3E0FAA3E0FBC374FF
:103BE200FF9BFF740F9AFEE499FDE498FCA3121761
:103BF200E6900CD3E0FCA3E0FDA3E0FEA3E0FFE42B
:103C0200FBFAF9F8D31217D55069E47FAA7E02FDB8
:103C1200FC900CD3E0F8A3E0F9A3E0FAA3E0FBC325
:103C22001217D5504E7F607EF07DFF7CFF900CD343
:103C3200E0F8A3A3A3E01216A2900CB21217E6902A
:103C42000CB2E0FCA3E0FDA3E0FEA3E0FFE47BAA4C
:103C52007A02F9F81258FD900CB21217E6900CB2E3
:103C6200E0FCA3E0FDA3E0FEA3E02428FFEE342362
:103C7200023CF5900CD3E0FCA3E0FDA3E0FEA3E040
:103C8200FFE47BAA7A02F9F8D31217D55072E4FF47
:103C92007E10FDFC900CD3E0F8A3E0F9A3E0FAA3B8
:103CA200E0FBC31217D550587F787EEC7DFF7CFF76
:103CB200900CD3E0F8A3A3A3E01216A2900CB212C8
:103CC20017E6900CB2E0FCA3E0FDA3E0FEA3E0FF48
:103CD200E47B567A0DF9F81258FD900CB21217E6F1
:103CE200900CB2E0FCA3E0FDA3E0FEA3E0246FFF92
:103CF200EE3417FEE43DFDE43CFC900CB21217E6F4
:103D0200900CB2E0FCA3E0FDA3E0FEA3E0FF900C68
:103D1200BA1217E6900CB2E0FCA3E0FDA3E0FEA30A
:103D2200E0FF900CBE1217E6900CC2E0FCA3E0FD8F
:103D3200A3E0FEA3E0FF900CAE1217E6900CAEE0FB
:103D4200FCA3E0FDA3E0FEA3E0FFE4FBFAF9F8D355
:103D52001217BF504DE4FF7E08FDFC900CAEE0F858
:103D6200A3E0F9A3E0FAA3E0FBC31217BF5033E4C8
:103D72007FF47E01FDFC900CAEE0F8A3A3A3E01259
:103D820016A2900CB21217E6900CB2E0FCA3E0FD72
:103D9200A3E0FEA3E0FFE4FB7A08F9F81258FD0263
:103DA2003EB4900CAEE0FCA3E0FDA3E0FEA3E0FF76
:103DB200E4FB7A08F9F8D31217BF506FE4FF7E0CC8
:103DC200FDFC900CAEE0F8A3E0F9A3E0FAA3E0FB5F
:103DD200C31217BF5055E47FDC7E05FDFC900CAE8C
:103DE200E0F8A3A3A3E01216A2900CB21217E69079
:103DF2000CB2E0FCA3E0FDA3E0FEA3E0FFE4FB7A4B
:103E020004F9F81258FD900CB21217E6900CB2E0C9
:103E1200FCA3E0FDA3E0FEA3E0243CFFEE34F6FEAB
:103E2200ED34FFFDEC34FFFC023EB4900CAEE0FC3E
:103E3200A3E0FDA3E0FEA3E0FFE4FB7A0CF9F8D3D4
:103E42001217BF5073E4FF7E10FDFC900CAEE0F839
:103E5200A3E0F9A3E0FAA3E0FBC31217BF5059E4B1
:103E62007F587E1BFDFC900CAEE0F8A3A3A3E012EA
:103E720016A2900CB21217E6900CB2E0FCA3E0FD81
:103E8200A3E0FEA3E0FFE47BFF7A03F9F81258FDFA
:103E9200900CB21217E6900CB2E0FCA3E0FDA3E096
:103EA200FEA3E024B3FFEE34B5FEED34FFFDEC34A7
:103EB200FFFC900CB21217E6900CBAE0F8A3E0F9FE
:103EC200A3E0FAA3E0FB900CB2E0FCA3E0FDA3E0C8
:103ED200FEA3E0FFEB2FFFEA3EFEE93DFDE83CFCDE
:103EE200900CBA1217E6900CC6E0FCA3E0FDA3E02A
:103EF200FEA3E0FF900CAE1217E6900CAEE0FCA31E
:103F0200E0FDA3E0FEA3E0FFE4FBFAF9F8D3121709
:103F1200BF504DE4FF7E08FDFC900CAEE0F8A3E03C
:103F2200F9A3E0FAA3E0FBC31217BF5033E47FF416
:103F32007E01FDFC900CAEE0F8A3A3A3E01216A252
:103F4200900CB21217E6900CB2E0FCA3E0FDA3E0E5
:103F5200FEA3E0FFE4FB7A08F9F81258FD02407272
:103F6200900CAEE0FCA3E0FDA3E0FEA3E0FFE4FBC7
:103F72007A08F9F8D31217BF506FE4FF7E0CFDFCEC
:103F8200900CAEE0F8A3E0F9A3E0FAA3E0FBC312C1
:103F920017BF5055E47FDC7E05FDFC900CAEE0F8C7
:103FA200A3A3A3E01216A2900CB21217E6900CB2D1
:103FB200E0FCA3E0FDA3E0FEA3E0FFE4FB7A04F94A
:103FC200F81258FD900CB21217E6900CB2E0FCA366
:103FD200E0FDA3E0FEA3E0243CFFEE34F6FEED3468
:103FE200FFFDEC34FFFC024072900CAEE0FCA3E05B
:103FF200FDA3E0FEA3E0FFE4FB7A0CF9F8D312176D
:10400200BF5073E4FF7E10FDFC900CAEE0F8A3E01D
:10401200F9A3E0FAA3E0FBC31217BF5059E47F589B
:104022007E1BFDFC900CAEE0F8A3A3A3E01216A247
:10403200900CB21217E6900CB2E0FCA3E0FDA3E0F4
:10404200FEA3E0FFE47BFF7A03F9F81258FD900C1F
:10405200B21217E6900CB2E0FCA3E0FDA3E0FEA3CF
:10406200E024B3FFEE34B5FEED34FFFDEC34FFFC8B
:10407200900CB21217E6900CBEE0F8A3E0F9A3E0B0
:10408200FAA3E0FB900CB2E0FCA3E0FDA3E0FEA3E8
:10409200E0FFEB2FFFEA3EFEE93DFDE83CFC900C21
:1040A200BE1217E6E47F167E03FDFC900CBAE0F820
:1040B200A3E0F9A3E0FAA3E0FB1216A2900CB61259
:1040C20017E6900CB6E0FCA3E0FDA3E0FEA3E0FF40
:1040D200E47B64FAF9F812172D900CB61217E6E495
:1040E2007FFF7EFFFDFC900CB6E0F8A3E0F9A3E0B1
:1040F200FAA3E0FBD31217D5400A900CB61217F2BE
:104102000000FFFF900CB6A3A3E0FEA3E0FDAC0607
:10411200900CD0E025E0FF900CCFE033FE744B2FE3
:10412200F58274003EF583ECF0A3EDF0E47F167E99
:1041320003FDFC900CBEE0F8A3E0F9A3E0FAA3E0D3
:10414200FB1216A2900CB61217E6900CB6E0FCA376
:10415200E0FDA3E0FEA3E0FFE47B64FAF9F81217A6
:104162002D900CB61217E6E47FFF7EFFFDFC900C4B
:10417200B6E0F8A3E0F9A3E0FAA3E0FBD31217D567
:10418200400A900CB61217F20000FFFF900CB6A383
:10419200A3E0FEA3E0FDAC06900CD2E025E0FF9088
:1041A2000CD1E033FE744B2FF58274003EF583ECA4
:0441B200F0A3EDF099
:1041B600900CADE004F07006900CACE004F0900CAE
:1041C600ACE07004A3E064066003023B1278AA7CAC
:1041D6000C7D017B017A00795F7E007F021215EC6F
:1041E600785F7C007D017B017A0079617E007F0229
:1041F6001215EC78617C007D017B017A0C79AA7E30
:06420600007F021215EC1E
:10420C00D007D006D005D004D003D002D001D00006
:0B421C00D0D0D082D083D0F0D0E032B0
:045C380043E810220B
:095C0C00758402D2ECE4F5842257
:104A4000900865E0FEA3E0FFEE6003024BA1EFB427
:104A500008004003024BA1904A5EF8282873024ADE
:104A600076024AA2024ACE024AFA024B25024B4380
:104A7000024B61024B7F78D87C0C7D017B017A0070
:104A8000795B7E007F021215EC78DA7C0C7D017B6D
:104A9000017A00794B7E007F021215EC903A4802B1
:104AA0004B9B78D87C0C7D017B017A00795D7E0080
:104AB0007F021215EC78DA7C0C7D017B017A00799B
:104AC0004D7E007F021215EC903A49024B9B78D83C
:104AD0007C0C7D017B017A00795F7E007F021215DC
:104AE000EC78DA7C0C7D017B017A00794F7E007FC7
:104AF000021215EC903A4A024B9B78D87C0C7D014F
:104B00007B017A0079617E007F021215EC78DA7CF5
:104B10000C7D017B017A0079517E007F021215EC39
:104B2000903A4B8076E4900CD8F0A3F078DA7C0CC5
:104B30007D017B017A007953FE7F021215EC903AD9
:104B40004C8058E4900CD8F0A3F078DA7C0C7D010E
:104B50007B017A007955FE7F021215EC903A4D8068
:104B60003AE4900CD8F0A3F078DA7C0C7D017B015C
:104B70007A007957FE7F021215EC903A4E801CE4C1
:104B8000900CD8F0A3F078DA7C0C7D017B017A00E0
:104B90007959FE7F021215EC903A4FE493900CD7AE
:104BA000F0E4F584C2FA900000E0F59B30FFFDC20E
:104BB000FFE4FFFE0FBF00010EEF64324E70F59070
:104BC0000CD7E0F59B30FFFDC2FFE4FEFF0FBF00F6
:104BD000010EEF64324E70F5900CD8E0F59B30FF7B
:104BE000FDC2FFE4FEFF0FBF00010EEF64324E7006
:104BF000F5900CD9E0F59B30FFFDC2FFE4FEFF0FFE
:104C0000BF00010EEF64324E70F5900000E0F59B9E
:104C100030FFFDC2FFE4FEFF0FBF00010EEF643264
:104C20004E70F5900CD7E0F59B30FFFDC2FFE4FE1F
:104C3000FF0FBF00010EEF64324E70F5900CDAE00A
:104C4000F59B30FFFDC2FFE4FEFF0FBF00010EEF3A
:104C500064324E70F5900CDBE0F59B30FFFDC2FF37
:104C6000E4FEFF0FBF00010EEF64324E70F5D2FA82
:014C70002221
:031A3000024C71F4
:104C7100C0E0C0F0C083C082C0D075D000C000C009
:0D4C810001C002C003C004C005C006C0078A
:104C8E0053E8DFAFBFEFFEADBE7C00E42DFFEC3E80
:104C9E00900023F0A3EFF0900023E0FCA3E0FD9042
:104CAE000863E0FF3395E0FEEF25E0FFEE33FE7480
:104CBE00262FF58274003EF583ECF0A3EDF09008FC
:104CCE0063E004F0C3648094885003024E5BE4F00A
:104CDE00900030E0FFA3E090000FCFF0A3EFF09034
:104CEE00002EE0FFA3E0900011CFF0A3EFF09000B4
:104CFE002CE0FFA3E0900013CFF0A3EFF090002A7A
:104D0E00E0FFA3E0900015CFF0A3EFF0900028E0B5
:104D1E00FFA3E0900017CFF0A3EFF0900026E0FF86
:104D2E00A3E0900019CFF0A3EFF090003EE0FFA3B8
:104D3E00E090001BCFF0A3EFF0900040E0FFA3E067
:104D4E0090001DCFF0A3EFF0900042E0FFA3E090A3
:104D5E00001FCFF0A3EFF0900044E0FFA3E090001F
:104D6E0021CFF0A3EFF0900001E06037E4FFEF25D4
:104D7E00E0240FF582E43400F583E0FCA3E0FDEFC0
:104D8E0025E0242FF582E4340DF583ECF0A3EDF04D
:104D9E000FEFB40AD9900001E004F0E0D3940F4075
:104DAE0002E4F0900001E070047D0180027D007F3E
:104DBE0000124227900001E070047D0180027D0008
:104DCE007F01124227900001E070047D0180027D78
:104DDE00007F02124227900001E070047D018002E4
:104DEE007D007F03124227900001E070047D018058
:104DFE00027D007F04124227900001E070047D01C5
:104E0E0080027D007F05124227900001E070047D34
:104E1E000180027D007F06124227900001E070049F
:104E2E007D0180027D007F07124227900001E07015
:104E3E00047D0180027D007F08124227900001E070
:104E4E0070047D0180027D007F0912422790086365
:034E5E00E0F5BBC1
:104E6100D007D006D005D004D003D002D001D000A5
:0B4E7100D0D0D082D083D0F0D0E0324F
:031A39000256F062
:1056F000C0E0C0F0C083C082C0D075D000C005C07B
:1057000006C007758402C2ED900025E5BEF0E07585
:10571000F010A4FD900864E0FF3395E0FEEF25E073
:10572000FFEE33FE74362FF58274003EF583E5F00C
:10573000F0A3EDF0900864E004F0C3648094884026
:1057400002E4F0900864E0F5BB758400D007D00651
:0D575000D005D0D0D082D083D0F0D0E03290
:1045820090003AE0FFA3E0900002CFF0A3EFF0909A
:10459200003CE0FEA3E0FF900004EEF0A3EFF0D3B6
:1045A200900007E09F900006E09E5016900004E005
:1045B200FFA3E0A3CFF0A3EFF090000AE4F0A3740E
:1045C20080F0900008E0FEA3E0FF900002E0FCA370
:1045D200E0FDC39FEC9E4011900008ECF0A3EDF0CB
:1045E20090000CE4F0A37480F0900047E024FF9266
:1045F20087900004E0FEA3E0FFD394A3EE94004072
:1046020003D38001C392B0D3EF94F4EE940040033D
:10461200D38001C392B1900004E0FEA3E0FFD394E3
:104622003BEE94024003D38001C392B2D3EF94D302
:10463200EE94034003D38001C392B3900004E0FEE2
:10464200A3E0FFD394BCEE94054003D38001C39250
:10465200B4D3EF9433EE940A4003D38001C392B5EE
:10466200D3900005E0944C900004E0940F4003D3F3
:104672008001C392B6D390000BE0940090000AE050
:1046820094004070900006E0FEA3E0FFD3944CEE4D
:10469200940F4004D2B6804CD3EF9433EE940A4088
:1046A20004D2B5803FD3EF94BCEE94054004D2B45B
:1046B2008032D3EF94D3EE94034004D2B38025D357
:1046C200EF943BEE94024004D2B28018D3EF94F4FC
:1046D200EE94004004D2B1800BD3EF94A3EE940089
:1046E2004002D2B090000BE024FFF090000AE034C8
:1046F200FFF08007E4900006F0A3F0900002E0FED5
:10470200A3E0FFD394A3EE94004003D38001C392AD
:10471200A0D3EF94F4EE94004003D38001C392A19E
:10472200900002E0FEA3E0FFD3943BEE940240032C
:10473200D38001C392A2D3EF94D3EE94034003D368
:104742008001C392A3900002E0FEA3E0FFD394BCD9
:10475200EE94054003D38001C392A4D3EF9433EEC9
:10476200940A4003D38001C392A5D3900003E0943E
:104772004C900002E0940F4003D38001C392A6D371
:1047820090000DE0940090000CE09400406F9000C7
:1047920008E0FEA3E0FFD3944CEE940F4004D2A6AF
:1047A200804CD3EF9433EE940A4004D2A5803FD3D9
:1047B200EF94BCEE94054004D2A48032D3EF94D39C
:1047C200EE94034004D2A38025D3EF943BEE9402EF
:1047D2004004D2A28018D3EF94F4EE94004004D2A5
:1047E200A1800BD3EF94A3EE94004002D2A09000DC
:1047F2000DE024FFF090000CE034FFF022E4900082
:0448020008F0A3F027
:01480600228F
:1055D40090086AE0A3F0E5B0548090086AF0A3E074
:1055E400FD90086AE0FE6D90000EF0EE703EED60F6
:1055F40007E490086CF0A3F090086DE004F07006E6
:1056040090086CE004F0D390086DE0948090086CEE
:10561400E09401404C900869E0700A900046E0FF75
:105624007D0C125B169008697401F02290086BE0FF
:10563400702FC390086DE094D090086CE0940050F3
:105644001B300409900047E06401F0800F9000478C
:10565400E06009A37401F0E4900047F0E490086965
:01566400F055
:015665002222
:105B5400900868E070051255D4800A900868E0B493
:0D5B64000103124582900868E06401F02200
:0614F400410D1200C105CC
:10566600125C1DE4900C73F0900C73E0FFC394067B
:105676005018EF25E02413F582E4340DF583E4F0A9
:10568600A3F0900C73E004F080DE900C737406F0C7
:10569600900C73E0FFC3940A501BEF25E02413F52A
:1056A60082E4340DF5837407F0A374FFF0900C7355
:1056B600E004F080DBE4900C73F0900C73E0FFC321
:1056C600941E502375F014EFA42401F582E5F034FE
:1056D60080AF82FE7C0D7D137B147A001258B79042
:0A56E6000C73E004F080D3025AA711
:1059ED00900C717402F0E4A3F0125C1D7E807F00B8
:1059FD007C0C7D717B017A001258B77E827F597CB9
:105A0D000C7D727B017A001258B7125AA7025666A6
:105B360030040F20050C900047E06006125C15D279
:0E5B46000522200408900047E0700204F022BF
:105BA600908259E493600C908000E4936402600351
:095BB6001259EDE4900D12F022E9
:105AF400900D12E075F014A42401F9748035F0FAC5
:105B04007BFF78137C0D7D017E007F141215ECC29F
:025B1400052268
:105AD000125C1D900D12E075F014A42401F582E50E
:105AE000F03480AF82FE7C0D7D137B147A00125857
:045AF000B7025AA7F8
:061A3300125AD0C2052288
:0A503800900C72EDF0900C71EFF097
:10504200D39B5003025116E024FFFEE434FF900C80
:1050520076F0A3CEF0EB14900C75F0900C72E02475
:10506200FFFFE434FFFE900C76E0FCA3E0FDD39F4B
:10507200EE6480F8EC64809840030251E79080016E
:1050820075F014ED121823EC75F014A42583AF8289
:10509200900C7DF0A3EFF0900C75E075F014A42451
:1050A20001F9748035F0FA900C7A74FFF0A3EAF0FB
:1050B200A3E9F0E4900C78F0A3F0900C7AA3E475E5
:1050C200F00112168CFEAFF0900C7DE475F0011227
:1050D200168C85F082F583E493FD12553E900C798F
:1050E200E004F07006900C78E004F0C3900C79E0D4
:1050F2009414900C78E0940040C0125AA7900C7758
:10510200E004F07006900C76E004F0900C75E00478
:10511200F002505D900C72E024FFFEE434FF900C2C
:1051220076F0A3CEF0900C74E014A3F0900C71E032
:1051320024FFFFE434FFFE900C76E0FCA3E0FDC305
:105142009FEE6480F8EC64809850030251E79080EF
:105152000175F014ED121823EC75F014A42583AF39
:1051620082900C7DF0A3EFF0900C75E075F014A422
:105172002401F9748035F0FA900C7A74FFF0A3EAF6
:10518200F0A3E9F0E4900C78F0A3F0900C7AA3E499
:1051920075F00112168CFEAFF0900C7DE475F001F3
:1051A20012168C85F082F583E493FD12553E900C25
:1051B20079E004F07006900C78E004F0C3900C796A
:1051C200E09414900C78E0940040C0125AA7900C1E
:1051D20077E024FFF0900C76E034FFF0900C75E05D
:0551E20014F002512E43
:0151E70022A5
:05188600900C71EDF073
:10188B00EF14900C8BF0EB14A3F0900C71E014FFA1
:10189B00900C8BE0D39F40030219E5A3E075F01485
:1018AB00A42401F582E5F03480AF82FEE4900C8D28
:1018BB00F0A3F0900C8DE0FCA3E0FDC39414EC942A
:1018CB0000502B0FEFAA0670010E14F5828A83E4E9
:1018DB0093FB74772DF582E4340CF583EBF0900CCD
:1018EB008EE004F070CD900C8DE004F080C5900C70
:1018FB008CE075F014A42401F9748035F0FA900C87
:10190B007274FFF0A3EAF0A3E9F0900C8BE075F092
:10191B0014A42401F582E5F03480AF82900C75F0AD
:10192B00A3EFF0E4900C8DF0A3F0900C72A3E47590
:10193B00F00112168CFEAFF0900C75E475F00112ED
:10194B00168C85F082F583E493FD12553E900C8E38
:10195B00E004F07006900C8DE004F0C3900C8EE068
:10196B009414900C8DE0940040C0900C8BE075F0BB
:10197B0014A42401F9748035F0FA900C7274FFF002
:10198B00A3EAF0A3E9F0E4900C8DF0A3F0900C8D9A
:10199B00E0FCA3E0FDC39414EC9400502D900C726A
:1019AB00A3E475F00112168CFEAFF074772DF5825F
:1019BB00E4340CF583E0FD12553E900C8EE004F000
:1019CB0070CB900C8DE004F080C3125AA7900C8B57
:0A19DB00E004F0A3E004F002189508
:0119E50022DF
:0751E800900C71EBF0AC0725
:1051EF00A2AFE433A3F0AF05A3E4F0A3EFF0E07FA9
:1051FF0000FE900C73F0A3EFF0AD04EDFF900C7375
:10520F00EEF0A3EFF0C2AF900C77E4F0A3740FF0C1
:10521F00125C1D900C77E0FEA3E0FF7C007D141262
:10522F00167A74012FF974803EFAA374FFF0A3EA83
:10523F00F0A3E9F0E4900C75F0A3F0900C73E0FC90
:10524F00A3E0FFECFD900C71E0FBE4900C80F0D23A
:10525F00021253B5900C7CEFF0FD900C79A3E4751E
:10526F00F00112168CFEAFF012553E900C74E00454
:10527F00F07006900C73E004F0900C76E004F07080
:10528F0006900C75E004F0C3900C76E09414900C2B
:10529F0075E0940040A5125AA7900C78E004F070C6
:1052AF0006900C77E004F0C3900C78E0941E900CFD
:1052BF0077E09400500302521F125941900C72E094
:0452CF0024FF92AF77
:0152D30022B8
:0752D400900C71EBF0AC0738
:1052DB00A2AFE433A3F0AF05900C77E4F0A3EFF0AB
:1052EB00E07F00FE900C77F0A3EFF0AD04EDFF90A4
:1052FB000C77EEF0A3EFF0C2AF900C75E4F0A37453
:10530B000FF0900C75E0FEA3E0FFC3941EEE94002B
:10531B0040030253A990800175F014EF121823EE8D
:10532B0075F014A42583AF82900C79F0A3EFF0E411
:10533B00900C73F0A3F0900C77E0FCA3E0FFECFD76
:10534B00900C71E0FB900C79E475F00112168C85D2
:10535B00F082F583E493900C80F0C2021253B59067
:10536B000C78E004F07006900C77E004F0900C746D
:10537B00E004F07006900C73E004F0C3900C74E042
:10538B009414900C73E0940040AC900C76E004F015
:10539B00600302530D900C75E004F002530D12598B
:0953AB0041900C72E024FF92AF66
:0153B40022D6
:1014FA00540D2F0000000000000000000000000052
:07150A0000000000000000DA
:1042270090FFFF121855EDF090FFFF121855EFF0B1
:0642370090FFEE12185585
:10423D00850883850982E4F0A3F0900012121879A5
:10424D00E025E0242FF582E4340DF583E0FEA3E0B4
:10425D00FFFBAA06E4F9F8900012121879E025E0A8
:10426D00240FF582E43400F583E0FEA3E0FFC3EFF5
:10427D009BFFEE9AFEE499FDE498FC850883850981
:10428D0082A3A31217E6E47F40FEFDFC850883851B
:10429D000982A3A3E0F8A3E0F9A3E0FAA3E0FBC32E
:1042AD001217BF400B850883850982E4F0A304F043
:1042BD0074FF7FC0FEFDFC850883850982A3A3E002
:1042CD00F8A3E0F9A3E0FAA3E0FBD31217BF500B5C
:1042DD0085088385098274FFF0A3F085088385091D
:1042ED0082E0FEA3E0FF4E700302457CEFF4700206
:0742FD00EEF4600302440926
:10430400900012121879E025E0242FF582E4340D90
:10431400F583E0FEA3E0FFE4FCFD90000E121879A3
:104324001217E6E47F01FEFDFC90000E121879E0FE
:10433400F8A3E0F9A3E0FAA3E0FBC31217BF500D02
:1043440090000E1218791217F2000000019000126A
:10435400121879E025E02413F582E4340DF583E0A6
:10436400FEA3E0FFE4FCFD7BFF7A0FF9F81216A22E
:1043740090000E121879E0F8A3E0F9A3E0FAA3E0A4
:10438400FB1258FD9000061218791217E6900012DD
:10439400121879E025E0240FF582E43400F583E077
:1043A400FEA3E0FFE4FCFD900006121879E0F8A3F8
:1043B400E0F9A3E0FAA3E0FB1216A290000A121897
:1043C400791217E6E47BFF7A0FF9F890000A1218C5
:1043D40079E0FCA3E0FDA3E0FEA3E0FF1258FD900A
:1043E4000012121879E025E02413F582E4340DF567
:1043F40083EEF0A3EFF0900013121879E07003023B
:0244040045531E
:10440600024550850883850982E0FEA3E064014EDB
:054416006003024553A4
:10441B00900012121879E025E02413F582E4340D94
:10442B00F583E0FEA3E0FBC374FF9BFF740F9EFEBE
:10443B00E49400FDE49400FCE47BFF7A0FF9F8129E
:10444B0016A29000061218791217E6900012121895
:10445B0079E025E0242FF582E4340DF583E0FEA30B
:10446B00E0FBC374FF9BFF740F9EFEE49400FDE41E
:10447B009400FC90000A1218791217E6E47F01FEF3
:10448B00FDFC90000A121879E0F8A3E0F9A3E0FA1A
:10449B00A3E0FBC31217BF500D90000A121879123C
:1044AB0017F200000001900006121879C083C08239
:1044BB00E0FCA3E0FDA3E0FEA3E0FF90000A1218CE
:1044CB0079E0F8A3E0F9A3E0FAA3E0FB1258FDD0E2
:1044DB0082D0831217E6900012121879E025E0249F
:1044EB000FF582E43400F583E0FEA3E0FBC374FF19
:1044FB009BFF740F9EFEE49400FDE49400FC90007F
:10450B0006121879E0F8A3E0F9A3E0FAA3E0FB1296
:10451B0016A2E47BFF7A0FF9F81258FDC374FF9FC4
:10452B00FF740F9EFE900012121879E025E0241301
:10453B00F582E4340DF583EEF0A3EFF09000131247
:08454B001879E06003125B36F1
:10455300900012121879E0FF25E0240FF582E4346D
:1045630000F583E0FCA3E0FDEF25E0242FF582E4D2
:09457300340DF583ECF0A3EDF02A
:06457C0090001402185526
:105B1600900CD7EFF0A3EDF07F0A125495900CD7B6
:105B2600E0FF125495900CD8E0FF125495021A0922
:085C15007F02125495021A09E6
:065A1D00125C2CEF602773
:105A2300900C71740DF0A37443F01259B7900C717C
:105A3300E475F00112168C85F082F583EFF0125CA9
:075A430032EF70E67F012243
:035A4A007F0022B8
:105BD500900C71EFF07F2F125495900C71E0FF122D
:055BE5005495021A09AD
:105BEA00900C71EFF07F30125495900C71E0FF1217
:055BFA005495021A0998
:0A151100410D1000410D1100C10151
:105B7100AF84E4F584C2C343E60243F60275C30170
:0B5B810075C04475CF8F43C3018F84B3
:015B8C0022F6
:105941007E0C7FE2900CE0EEF0A3EFF0900CDEEE27
:10595100F0A3EFF0900CDCEEF0A3EFF07E0C7FFCF7
:10596100900CFAEEF0A3EFF0900CF8EEF0A3EFF04C
:0D597100900CF6EEF0A3EFF0C200025B71A7
:10597E00900CDEE475F00112168C85F082F583EF43
:10598E00F0900CDEE475F00112168C85F082F58332
:10599E00EDF0900CDEE0B40C0FA3E0B4F60A900C20
:0959AE00DE740CF0A374E2F02297
:0D1A0900AF84E4F584C200C2C4D2C58F844E
:011A160022AD
:10549500200055D200900CF8E475F00112168C85A9
:1054A500F082F58374FFF07C0D7D10900CF8E0B56B
:1054B500040FA3E0B5050A900CF8740CF0A374FC76
:1054C500F0900CF8E475F00112168C85F082F583E6
:1054D500E4F0900CF8E0B5040FA3E0B5050A900CD4
:1054E500F8740CF0A374FCF0900CF8E475F001125C
:1054F500168C85F082F583E4F0900CF8E0B40D0F7E
:10550500A3E0B4100A900CF8740CF0A374FCF090AE
:105515000CF8E475F00112168C85F082F583EFF036
:10552500900CF8E0B40D0FA3E0B4100A900CF874D9
:095535000CF0A374FCF07F0122CC
:105A7B00900CE0E0FCA3E0FD900CDCE0B50408A387
:105A8B00E0B505037F0022900CE0E0FCA3E0F5827B
:0C5A9B008C83E0B507037F01227F00220E
:1059B700900CE1E004F07006900CE0E004F0900C2D
:1059C700E0E475F00112168C85F082F583E0FF9014
:1059D7000CE0E0B40C0FA3E0B4F60A900CE0740CF2
:0559E700F0A374E2F0E2
:0159EC002298
:065C2C007FFF125A7B22EB
:065C3200E4FF125A7B2280
:031A18000248077A
:10480700C0E0C0F0C083C082C0D075D000C000C077
:1048170004C005C006C007E5C154F812182F49FCAB
:104827000048620848621048B01848FC2049092827
:1048370049943049A03849B15049B15849C46049F1
:10484700B36849C47049B37849B18049D38849B13D
:104857009049D39849E4A000004A29C2C5900CF7B3
:10486700E004F07006900CF6E004F07E0D7F1090E7
:104877000CF6E0B5060FA3E0B5070A900CF6740C2A
:10488700F0A374FCF0900CF6E475F00112168C8519
:10489700F082F583E0F5C2900CF6E06E7003A3E0BA
:1048A7006F6003024A29024987900CF7E004F07011
:1048B70006900CF6E004F07E0D7F10900CF6E0B544
:1048C700060FA3E0B5070A900CF6740CF0A374FC6E
:1048D700F0900CF6E475F00112168C85F082F583E2
:1048E700E0F5C2900CF6E06E7003A3E06F60030280
:1048F7004A29024987900CFAE0FFA3E0900CF6CF13
:10490700801B900CF8E0FEA3E0FF900CF6E0FCA300
:10491700E0FDB50713ECB5060F900CFAEEF0A3EF28
:10492700F0C2C5D2C4024A298D828C83E0B4FF0746
:10493700C2C4D2C5024A29900CF7E004F070069071
:104947000CF6E004F07E0D7F10900CF6E0B5060F34
:10495700A3E0B5070A900CF6740CF0A374FCF09072
:104967000CF6E475F00112168C85F082F583E0F5FC
:10497700C2900CF6E06E7003A3E06F6003024A2951
:10498700900CF6740CF0A374FCF0024A29900CFA10
:10499700E0FFA3E0900CF6803B900CFAE0FFA3E069
:1049A700900CF6CFF0A3EFF080788017900CFAE028
:1049B700FFA3E0900CF6CFF0A3EFF0D201ADC27FDA
:1049C700FF8004ADC2E4FF12597E8056900CDCE0F4
:1049D700FFA3E0A3CFF0A3EFF0D2C48045900CDE95
:1049E700E0FFA3E0900CDCCFF0A3EFF0300133D26F
:1049F700C5C201802D900CFAE0FEA3E0FF900CF6F3
:104A0700EEF0A3EFF0900CDCE0FDA3E0A3CDF0A364
:104A1700EDF0D2C4900CF8E06E7003A3E06F600273
:104A2700D2C5C2C3D007D006D005D004D000D0D09D
:094A3700D082D083D0F0D0E0322F
:10586B00900C96E584F0A2AF9202AF01AE027C00E1
:10587B00E4FDA31217E6900C99E0FEA3E0780AA6CC
:10588B000608F6E4F584C2AF43B701438F02438F9A
:10589B000118E6FE08E6F5828E83E4F053B7FEF5B9
:0B58AB008FA20292AF900C96E0F584F3
:0158B60022CF
:0557C200900C9CEDF0CD
:1057C700A3E584F0A2AF9202AF01AE027C00E4FD34
:1057D700A31217E6900C9CE0FFFD3395E0FCEDF477
:1057E7004C6029900CA0E0FCA3E0780AA60408F618
:1057F700E4F584C2AF43B701758F0118E6FC08E6EC
:10580700F5828C83EFF053B7FEE4F58FA20292AFD7
:06581700900C9DE0F584F9
:01581D002268
:10575D00900C96EEF0A3EFF0A3ECF0A3EDF0A3EA1E
:10576D00F0A3EBF0900C9AE07002A3E06046900C71
:10577D0096E0FEA3E0AA06F97B01A3E0FEA3E0F507
:10578D00828E83E0FD1257C2900C9BE024FFF090B7
:10579D000C9AE034FFF0900C99E004F07006900C38
:1057AD0098E004F0900C97E004F070B8900C96E03F
:0557BD0004F080B022A1
:085C1D00E4900C6EF0A3F022EC
:105AA700900C6EE0FEA3E0AA06F97B0112586B90FA
:105AB7000C6EE0FEA3E0FF7C087D6E1B7A04125794
:095AC7005DE4900C6EF0A3F022E6
:0D553E00900C91EDF0900C8FEEF0A3EFF0CB
:10554B00EE54FCFE900C6EE0FCA3E0FD7002EE6CE2
:10555B006059ED4C6003125AA7900C8FE0FEEE548D
:10556B00FCFE7F00900C6EF0A3EFF0900C92EEF02F
:10557B00A3EFF0A37408F0A3746EF07FFF7E03908B
:10558B000C92E475F00112168C85F082F583E4938E
:10559B00FD900C94E475F00112168C85F082F58366
:1055AB00EDF0EF1F70011EEF4E70D4900C91E0FFE9
:1055BB00900C8FE0FCA3E0FDEC5403FC746E2DF516
:0855CB008274083CF583EFF047
:0155D30022B5
:1058B700900C74EEF0A3EFF0A3ECF0A3EDF0A3EAE5
:1058C700F0A3EBF0900C7874FFF5F012168C45F00E
:1058D7006023900C74E475F00112168CAFF0FE9003
:1058E7000C76E475F00112168C85F082F583E0FDE5
:0658F70012553E80CF2295
:0753B500900C7DEFF0A9054B
:1053BC00C20320C3FD20C5FAC2C4D2C5E4FFFD3030
:1053CC00C3FD30C3FDE5C154F8FC64086004ECB4C3
:1053DC001013EFB40105EB44018003EB54FEF5C24E
:1053EC007D01025483ECB4180B89C27D02C2C4C285
:1053FC00C5025483ECB420028045EC6428703CED6B
:10540C00B4020E900C7DE0F5C27D03C2C5C2C4800F
:10541C0066EDB4031B300208D2C57F01C2C48057AD
:10542C00900C80E0F5C2C2C57D04E4FFC2C4804785
:10543C00ED64047042D2C47D05803CECB4300AD2D9
:10544C00C4D2C57D08E4FF802EECB438028024EC75
:10545C00B44006C2C2C2C5801EECB448028014EC33
:10546C00B450028004ECB4580AD2C47D07AEC2C258
:10547C00C28004D2C4D2C5C2C3ED64076008ED6417
:08548C000560030253CEAF06D8
:0154940022F5
:100C1A00024E7CE493A3F8E493A34003F68001F226
:100C2A0008DFF48029E493A3F85407240CC8C333DB
:100C3A00C4540F4420C8834004F456800146F6DFAA
:100C4A00E4800B0102040810204080900C9AE47E94
:100C5A00019360BCA3FF543F30E509541FFEE4939F
:100C6A00A360010ECF54C025E060A840B8E493A366
:100C7A00FAE493A3F8E493A3C8C582C8CAC583CA91
:100C8A00F0A3C8C582C8CAC583CADFE9DEE780BE49
:01151B0000CF
:10151C00E709F608DFFA8046E709F208DFFA803EB1
:10152C0088828C83E709F0A3DFFA8032E309F6089E
:10153C00DFFA8078E309F208DFFA807088828C8306
:10154C00E309F0A3DFFA806489828A83E0A3F608BA
:10155C00DFFA805889828A83E0A3F208DFFA804C94
:10156C0080D280FA80C680D4806980F2803380106B
:10157C0080A680EA809A80A880DA80E280CA8033D4
:10158C0089828A83ECFAE493A3C8C582C8CCC5834C
:10159C00CCF0A3C8C582C8CCC583CCDFE9DEE7801C
:1015AC000D89828A83E493A3F608DFF9ECFAA9F09B
:1015BC00EDFB2289828A83ECFAE0A3C8C582C8CCF1
:1015CC00C583CCF0A3C8C582C8CCC583CCDFEADE0A
:1015DC00E880DB89828A83E493A3F208DFF980CC6C
:1015EC0088F0EF60010E4E60C388F0ED2402B40465
:1015FC000050B9F582EB2402B4040050AF2323450C
:06160C00822390156C73AF
:10161200C2D530F707B2D563F0FF05F030E70CB260
:10162200D5F4048463F0FF05F080018430D502F420
:02163200042290
:10163400BB010689828A83E0225002E722BBFE02B4
:09164400E32289828A83E49322E7
:10164D00BB010CE58229F582E5833AF583E0225052
:10165D0006E92582F8E622BBFE06E92582F8E2229C
:0D166D00E58229F582E5833AF583E49322B6
:10167A00EF8DF0A4A8F0CF8CF0A428CE8DF0A42E84
:02168A00FE223E
:10168C00A3F8E0C5F025F0F0E58215827002158311
:06169C00E0C838F0E8226E
:1016A200E88FF0A4CC8BF0A42CFCE98EF0A42CFCE7
:1016B2008AF0EDA42CFCEA8EF0A4CDA8F08BF0A465
:1016C2002DCC3825F0FDE98FF0A42CCD35F0FCEBC4
:1016D2008EF0A4FEA9F0EB8FF0A4CFC5F02ECD3989
:0F16E200FEE43CFCEAA42DCE35F0FDE43CFC22F6
:1016F10075F008758200EF2FFFEE33FECD33CDCCB0
:1017010033CCC58233C5829BED9AEC99E582984032
:101711000CF582EE9BFEED9AFDEC99FC0FD5F0D60F
:10172100E4CEFBE4CDFAE4CCF9A88222B800C1B939
:101731000059BA002DEC8BF084CFCECDFCE5F0CB77
:10174100F97818EF2FFFEE33FEED33FDEC33FCEBB0
:1017510033FB10D703994004EB99FB0FD8E5E4F96B
:10176100FA227818EF2FFFEE33FEED33FDEC33FC58
:10177100C933C910D7059BE99A4007EC9BFCE99A4C
:10178100F90FD8E0E4C9FAE4CCFB2275F010EF2F91
:10179100FFEE33FEED33FDCC33CCC833C810D70791
:1017A1009BEC9AE899400AED9BFDEC9AFCE899F8CC
:0E17B1000FD5F0DAE4CDFBE4CCFAE4C8F9225F
:1058FD00C2D5E830E70FB2D5E4C39BFBE49AFAE4D6
:10590D0099F9E498F8EC30E717B2D512593312171C
:10591D002DE4C39BFBE49AFAE499F9E498F880032B
:10592D0012172D30D50DE4C39FFFE49EFEE49DFDBF
:04593D00E49CFC22C8
:1017BF00EB9FF5F0EA9E42F0E99D42F0EC6480C8A1
:0617CF0064809845F02241
:1017D500EB9FF5F0EA9E42F0E99D42F0E89C45F06A
:0117E50022E1
:0C17E600ECF0A3EDF0A3EEF0A3EFF02276
:1017F200A8828583F0D083D08212180912180912A8
:101802001809121809E473E493A3C583C5F0C583CC
:10181200C8C582C8F0A3C583C5F0C583C8C582C840
:0118220022A3
:0C182300A42582F582E5F03583F58322D0
:10182F00D083D082F8E4937012740193700DA3A348
:10183F0093F8740193F5828883E47374029368605C
:06184F00EFA3A3A380DF5C
:10185500E5092582F582E5083583F583B508048514
:1018650082092210AF06858209F50822858209F5CD
:0418750008D2AF22C4
:0D187900E5092582F582E5083583F5832217
:00000001FF
